:020000040000FA
:100000000508A2000608A3001D288312C800CE011F
:100010001828831203131630A0002C30A1000A12F6
:100020008A11A10B0F280A128A11A00B0D28CE0AE3
:100030004E084802031D09280800BC014414C410DE
:100040004411C4159828C800613048024F10031DA0
:1000500003184F147A304802CF10031D031CCF142D
:100060004F154F18CF1C4F114F1D3C2861304802CF
:10007000CE0041304E07C80048080800C8004808B4
:10008000BF3E0318F93E113EC80048080800EE00C4
:100090006E08F63E0318073E3A3EEE006E08080072
:1000A0008312E700E8017D282808A7002908A80096
:1000B0002A08A9002B08AA002C08AB002D08AC00C8
:1000C0002E08AD002F08AE003008AF003108B00098
:1000D0003208B1003308B2003408B3003508B40068
:1000E0003608B5003708B6003808B7003908B80038
:1000F0003A08B9003B08BA00E80A68086702031D1D
:100100005428080083124416221222088500080091
:100110008312441222162208850008008312C4129A
:10012000441AC41608008312C41E972882288828FF
:1001300044138A151B2E4419A42883160610831213
:10014000C41DA42883168611831222152208850057
:1001500044170800831606148615831222112208FC
:1001600085004413080083122310C41B23142308A2
:100170008600C41FBD28C413BE28C417A311C41B06
:10018000A31523088600080083122310C41B231420
:1001900023088600C41FCE28C413CF28C417A31178
:1001A000C41BA31523088600000000000000000007
:1001B00008008316A400A501E928A601C4208A111D
:1001C000C4208316A60A0A3026028A11031DDE28DF
:1001D000A50A25082402031DDD2808008316A300B4
:1001E000A401FE28A501C4208A11C4208316A50AF3
:1001F000643025028A11031DF328A40A240823026F
:10020000031DF2280800231C0E29831244180B2911
:100210008316A31016298316A31416298312C41853
:1002200014298316A31016298316A3148E208A116D
:100230008820831623118A11231C23298312441D2D
:100240002329831623158316231929298312A3131F
:100250002B298312A3172308860083168613A3185D
:100260003429831223133629831223172308860087
:1002700083160613A3183F298312A2114129831262
:10028000A21522088500A214220885003230D92048
:100290008312A2102208850032308A11D9208316D9
:1002A000861706178312A2112208850032308A11A0
:1002B000D9208A1193288312441F62290A30EE2024
:1002C0008A1166299B20C8308A11EE208312A2145D
:1002D00022088500221022088500A3122308860028
:1002E00083160510861223148A1103290514861615
:1002F0008312A21422088500441F8229AA20C83034
:100300008A11EE2083162310201823148A11032942
:100310008316201076298316201476298312DB0099
:1003200024308316980083125B088316990090305E
:10033000831298008316861406110800831686140B
:10034000061183122315230886008316980199014C
:10035000831298010800831220100C1A2014080040
:10036000DB00AB2183125F1020185F148A115F1825
:10037000BC29B3208A11B1295B08990008008312B7
:100380009810181DC8298618C629C32940308E2107
:10039000831220108C1A201408001A0808008316F3
:1003A000A9008612AB01EC292918D9298312A312BE
:1003B000DB298312A3162308860022142208850055
:1003C00003108316A90CB320831222102208850083
:1003D0008A11B3208316AB0A2B082A028A11031D47
:1003E000D429C4288312EE0083168616A001092A98
:1003F000221422088500B32003108312EF0CEF13A0
:10040000861AEF172210220885008A11B32083165E
:10041000A00A200883126E028A11031DF829C42045
:1004200083126E098316A1000930A1072108FE007E
:1004300083126F088316A200FE088A110319242A6A
:100440000310A20CFE0B202A220808008312E800E9
:100450006808F2218312E9000F306905EA006A0892
:100460008A1147288316A4000630AA002408CF2941
:10047000A0000130AA000030CF2108308316AA0066
:1004800021088A11CF2106308316AA0020088A117C
:10049000CF2101308316AA0000308A11CF29A6008F
:1004A0000430AA002608CF2108308316AA002808A5
:1004B0008A11CF2108308316AA0027088A11CF2974
:1004C0008312E70004308316AA0083126708CF2145
:1004D00008308A11F22108308A11F229033083167C
:1004E000AA000030CF218312A31223088600221411
:1004F000220885003D088A11D92083122210220883
:1005000085008A11C42010308316AA0000308A1199
:10051000CF290E308316A700831241088316A80046
:1005200000304F226E308316A700F830A80000304C
:100530008A114F220E308316A700831240088316BB
:10054000A80000308A114F226E308316A700F730C2
:10055000A80000308A114F220E308316A7008312A4
:100560003F088316A80000308A114F226E30831690
:10057000A700F630A80000308A114F2A8312E80045
:10058000E901CF2AB3208312BF0A3F088A11031D55
:10059000CE2AC00A4008031DCE2AC10AE90A69080A
:1005A0006802031DC22A08008316A30023088312D1
:1005B000C100831624088312C00083162508831205
:1005C000BF00892A8E308316A700A630A80000300D
:1005D0004F228C308316A700A630A80000308A1165
:1005E0004F228316A4010630A5003C308A11D42284
:1005F0008316A701A8010C308A114F2AA0002008F9
:10060000322201308316AA0000308A11CF21043033
:100610008316AA0083123B088A11CF210430831667
:10062000AA0083123A088A11CF2104308316AA0047
:10063000831239088A11CF2102308316AA0083124F
:1006400038088A11CF2101308316AA0000308A11A0
:10065000CF21831621088A11322283123D088A1184
:10066000D920831623088A110319382B2308322A2C
:100670000800A0005B218316A4010530A5003C30D2
:100680008A11D42283162008A7002008A8000C3065
:100690008A114F228316A4010430A5003C308A1130
:1006A000D42283162108A7002108A8000C308A1143
:1006B0004F228316A701A80100308A114F2204306F
:1006C0008316AA0000308A11CF2106308A11EE204D
:1006D00010308316AA0000308A11CF29822083129D
:1006E0002508A600BC010130BE00380EF039CE004E
:1006F0004E083907BD00C101C001BF010A303B02ED
:100700008A11031D862B88208A118B290B303B020E
:10071000031D972B4410BA184414C4103A19C4147A
:1007200044113A184415C411BA19C41508000C3004
:100730003B02031D612C3A08CF15031DCF11053074
:100740003A024F1203194F16CF12CF1D4F1ACF1670
:10075000CF1EB82B0130BC006430C8005B210530CF
:1007600083123A028A11031D282F0430BE00282F5D
:1007700001303A02031DC32B0330BC000A30C8000D
:100780005B218A11282F02303A02031DCE2B05303F
:10079000BC000A30C8005B218A11282F03303A02BE
:1007A000D0100319D01406303A0250110319501515
:1007B000D011D01C5019D01509303A02501203192B
:1007C0005016D012D01D501AD016D01E0D2C32301B
:1007D000BC000A30C8005B218A11E2228E308316E9
:1007E000A700A630A80000308A114F229C30831643
:1007F000A700A630A80000308A114F228316A4015A
:10080000A50100308A11D422063083123A028A11DF
:10081000031D602C0830BE00282F04303A02031D4F
:10082000182C0130BC005030C8005B218A11282FE1
:1008300007303A0251100319511408303A02D1100E
:100840000319D1145111511CD1185115511D2F2CC0
:100850000730BC000A30C8005B218A11282F0B30FA
:100860003A02031D3A2C0930BC001430C8005B2149
:100870008A11282F0A303A02031D482C0B30BC0085
:100880001430C8005B2106308A1132228A11282FC9
:100890000C303A02031D532C0C30BC001930C80038
:1008A0005B218A11282F0D303A02031D5E2C0E3079
:1008B000BC001930C8005B218A11282F3F30A600E8
:1008C000282F0D303B02031DF72C2130C0003A08C1
:1008D0005214031D521008303A02D2100319D214D8
:1008E0005211521CD2185215521D7D2C0230BC00E0
:1008F0006430C8005B218A11282F01303A02031DA1
:10090000882C0430BC006430C8005B218A11282F79
:1009100002303A0252120319521607303A02D2122A
:100920000319D2165213521ED21A5217521F9F2C5D
:100930000630BC006430C8005B218A11282F0C30BF
:100940003A02031DAA2C0D30BC006430C8005B21A4
:100950008A11282F03303A0253100319531406301A
:100960003A02D3100319D3145311531CD31853153F
:1009700009303A02D3110319D3155312531DD31959
:100980005316531EE92C3330BC000A30C8005B21DB
:100990008312C0019E308316A700A630A800003045
:1009A0008A114F229C308316A700A630A800003081
:1009B0008A114F22063083123A028A11031DE22C5B
:1009C0000830BE0009303A02031DF62C3530BC0059
:1009D000282F04303A02031DF42C5030C800023096
:1009E000BC005B218A11282F3F30A600282F0F3032
:1009F0003B02031DD72D2030C0003A08D414031D3C
:100A0000D41001303A02541103195415D411D41CD6
:100A10005419D41502303A02541203195416D41240
:100A2000D41D541AD41604303A025413031954171F
:100A3000D413D41E541BD41707303A02551003198F
:100A40005514D510D41F5518D51408303A02551135
:100A500003195515D511D51C5519D5150B303A026A
:100A6000551203195516D512D51D551AD5160C3029
:100A70003A02551303195517D513D51E551BD51713
:100A80000D303A02561003195614D610D51F5618B9
:100A9000D614D61C812D0130BC005B2100308A1198
:100AA00032228316A10100308A1138226430831269
:100AB000C80002303A0256110319561507303A029F
:100AC000D6110319D6155612561DD61956168A1167
:100AD000561E6C2D0530BC0001303A02031D722DEC
:100AE0000330BC000C303A02031D7A2D0C30BC00E0
:100AF0003230C8000D303A02031D282F0E30BC00E2
:100B0000282F03303A0257100319571406303A02BF
:100B1000D7100319D7145711571CD7185715093078
:100B20003A02D7110319D7155712571DD71957165F
:100B3000571EBE2D3430BC005B218E308316A700BB
:100B4000A630A80000308A114F228C308316A700EF
:100B5000A630A80000308A114F228316A401A501F7
:100B600030308A11D4220A308312C80006303A028B
:100B70008A11031D282F0830BE00282F0A303A02A0
:100B8000031DC92D0B30BC001430C8005B218A1135
:100B9000282F0D303A02031DD42D0F30BC00143025
:100BA000C8005B218A11282F3F30A600282F0E3065
:100BB0003B02031D262F3A08031D232E5B21003024
:100BC0008A113222FF308316A1003F308A11382269
:100BD0008312EF0106308A1132228312EF0A0730A6
:100BE0006F028A11031DEA2D0130322207308A116B
:100BF000322208308A1132220A308A11EE20013066
:100C00008A11322207308A113222831623148A1164
:100C1000032103308A113222FF308316A1000030F5
:100C20008A11382208308A1132220A308A11EE20C5
:100C30000B308A11322208308A1132220A308A118E
:100C4000EE208A11282F01303A02031D382E5B2135
:100C500000308A1132228316A10100308A11382215
:100C600009308A11322232308A11EE208A11282F5F
:100C700002303A0258120319581607303A02D812B5
:100C80000319D8165813581ED81A5817581F592E1A
:100C90005B2100308A1132228316A10100308A11B3
:100CA00038221F308A11322205308A11EE208A1133
:100CB000282F04303A02D8130319D8170B303A0200
:100CC000591003195914D910D81F5918D914D91CFF
:100CD000812E5B2100308A113222FF308316A10061
:100CE0003F308A11382209308A1132220A308A11A3
:100CF000EE200B308A1132220A308A11EE208A113E
:100D0000282F08303A02031DA32E5B2100308A11E0
:100D10003222FF308316A1003F308A113822093079
:100D20008A1132220A308A11EE2009308A113222C9
:100D30000A308A11EE200B308A1132220A308A11D1
:100D4000EE208A11282F0C303A02031DBE2E5B21A3
:100D500000308A1132228316A10100308A11382214
:100D600009308A11322206308A11EE200B308A11A6
:100D7000322206308A11EE208A11282F03303A02DF
:100D8000031DE82E5B218316A4010430A5003C302E
:100D90008A11D4228316A7018030A8000C308A1152
:100DA0004F228316A701A80100308A114F22043078
:100DB0008316AA0000308A11CF2106308A11EE2056
:100DC00010308316AA0000308A11CF218A11282FF3
:100DD00009303A02031DF92E8F308316A1003F30EF
:100DE000392387308316A1000F308A1139238A11E5
:100DF000282F0A303A02031D062F5B2109308A1181
:100E0000322214308A11EE208A11282F0D303A0236
:100E1000031D232F5B218312EF0106308316A100EF
:100E20000630A30000308A11FE228312EF0A04303C
:100E30006F028A11031D0D2F0930322214308A11DE
:100E4000EE208A11282F3F30A600282F3F30A60021
:100E500083123D08031D2E2F4808BD0008003230C4
:100E60003C0203193C2F03183C2F2508A60006302E
:100E7000322201308A11BE2A3F30A6000800E70066
:100E80006708322201308A11F22104308A112622A9
:100E90008312BB0004308A1126228312BA00043068
:100EA0008A1126228312B90002308A112622831267
:100EB000B80001308A11F2291030C8002508A600B8
:100EC00032303C020319662F031C682F1230C80011
:100ED000CE018A15A72801303C02DB100319DB1470
:100EE00003303C025B1103195B15DB11DB1C5B1942
:100EF000DB1505303C025B1203195B16DB12DB1DB0
:100F00005B1ADB1607303C025B1303195B17DB131C
:100F1000DB1E5B1BDB1709303C025C1003195C1401
:100F2000DC10DB1F5C18DC140B303C025C11031975
:100F30005C15DC11DC1C5C19DC150C303C025C120D
:100F400003195C16DC12DC1D5C1ADC160E303C0248
:100F50005C1303195C17DC13DC1E5C1BDC17DC1F45
:100F6000C42F04303F27013083123E028A11031937
:100F7000BC2F031CBC2F2F2704308A1150200430B3
:100F80008312C8028A15A62802303C02DD1003191C
:100F9000DD1404303C025D1103195D15DD11DD1C0B
:100FA0005D19DD1506303C025D1203195D16DD1278
:100FB000DD1D5D1ADD160D303C025D1303195D1752
:100FC000DD13DD1E5D1BDD17DD1FF52F05303F270F
:100FD00030308312B8003030B90004308A1150200C
:100FE00004308312C8028A15A62832303C025E10F3
:100FF00003195E1434303C02DE100319DE145E1156
:101000005E1CDE185E158A155E1D262809308A11C1
:1010100060228312E600660E0F39CF004F088A1156
:1010200047208312BA000F306605CF004F088A119F
:1010300047208312BB0001308A11BE2202308A1180
:10104000502002308312C8028A15A62833303C0291
:10105000DE110319DE1535303C025E1203195E16EF
:10106000DE12DE1D5E1ADE16DE1EA4280E3083168A
:10107000A70083123F088316A80000308A114F2270
:101080006E308316A700A930A80000308A114F22C5
:101090000E308316A700831240088316A800003084
:1010A0008A114F226E308316A700AA30A8000030A4
:1010B0008A114F2280308316A700A630A800003086
:1010C0008A114F2250308316A700A830A8000030A4
:1010D0008A114F226E308316A700F530A800003029
:1010E0008A114F22353083123C028A15031D842851
:1010F0008316A701A80100308A114F228316A70189
:10110000A80100308A114F2202308A116022831216
:10111000E600660E0F39CF004F088A114720831270
:10112000BA000F306605CF004F088A11472083129E
:10113000BB0001308A11BE2202308A1150200230D9
:101140008312C8028A15A6283F30A600CE0A4E0890
:101150003E028A11031D6B2F480850288A118220F5
:1011600083122508A60001303C028A15031DBF2802
:1011700008308316A100A30102308A11FE2A023032
:101180003C02031DCA2808308316A100A3010330C6
:101190008A11FE2A03303C02031DD628083083162C
:1011A000A1000E30A30002308A11FE2A04303C0256
:1011B000031DDD283F30A600080005303C02031D5A
:1011C000E92818308316A1001730A30002308A11D5
:1011D000FE2A06303C02031DF52818308316A100B4
:1011E0001730A30003308A11FE2A0D303C02031D84
:1011F000012918308316A1000A30A30003308A1198
:10120000FE2A0E303C02031D0D2918308316A10062
:101210000A30A30002308A11FE2A0F303C02031D5F
:10122000192918308316A1000A30A30000308A1152
:10123000FE2A07303C02E0100319E01408303C029B
:10124000601103196015E011E01C6019E015093008
:101250003C02601203196016E012E01D601AE016ED
:10126000E01E96290430E700670803198629E70382
:1012700002308A11322201308316AA0000308A110E
:10128000CF2104308316AA0083122F088A11CF21A0
:1012900004308316AA0083122E088A11CF2104304D
:1012A0008316AA0083122D088A11CF2102308316DB
:1012B000AA0083122C088A11CF2101308316AA00BC
:1012C00000308A11CF21831267088A1503196B2910
:1012D00006308A11322283123008AC003408B00084
:1012E0003808B4003108AD003508B1003908B50040
:1012F0003208AE003608B2003A08B6003308AF0034
:101300003708B3003B08B7008A15342918308A1112
:10131000322283123D088A11D92017308A113222D5
:1013200006308A11322204308A11BE2A08303C026B
:10133000031DA22908308316A1000E30A30002303D
:101340008A11FE2A0C303C02031DAD290830831699
:10135000A100A30102308A11FE2A0B303C02031DBA
:10136000B92908308316A1000E30A30002308A117B
:10137000FE2A32303C02031D202A8A118922831260
:101380002E0EF039C8002F084807C9002C0EF0397E
:10139000CA002D084A07CB0049088316A70083120C
:1013A0004B088316A8000D308A114F228312320E8B
:1013B000F039C80033084807C900300EF039CA00B8
:1013C00031084A07CB0049088316A70083124B084F
:1013D0008316A8000D308A114F228312360EF03981
:1013E000C80037084807C900340EF039CA0035086C
:1013F0004A07CB0049088316A70083124B088316BF
:10140000A8000D308A114F2283123A0EF039C8001D
:101410003B084807C900380EF039CA0039084A07A6
:10142000CB0049088316A70083124B088316A80037
:101430000F308A114F228A116E2208308A11BE2A7B
:1014400033303C0261120319611635303C02E1125F
:101450000319E1166113611EE11A6117611FD92A90
:101460000E308316A70083123F088316A8000030B1
:101470008A114F226E308316A700A930A8000030D1
:101480008A114F220E308316A7008312400883165C
:10149000A80000308A114F226E308316A700AA30B0
:1014A000A80000308A114F2283123A0EF039C8008A
:1014B0003B084807C9000E308316A700831249086D
:1014C0008316A80000308A114F226E308316A700C1
:1014D000A830A80000308A114F2284308316A7005C
:1014E000A630A80000308A114F22333083123C020C
:1014F0008A15031D9B2A0E308316A7005530A800BD
:1015000000308A114F226E308316A700A730A80042
:1015100000308A114F220E308316A700AA30A8008F
:1015200000308A114F226E308316A700A730A80022
:1015300000308A114F2282308316A700A630A800FF
:1015400000308A114F2250308316A700A630A80021
:1015500000308A114F226E308316A700F530A800A4
:1015600000308A114F22353083123C028A15031D48
:10157000BF2A8316A701A80100308A114F22043028
:101580008316AA0002308A11CF2106308A11EE207C
:1015900010308316AA0000308A11CF2194308316B0
:1015A000A700A630A80000308A114F2201308A110E
:1015B000BE2A34303C02031DF52A8A118922831287
:1015C0003A0EF039C8003B084807E7006708831661
:1015D000A700831267088316A8000F308A114F22D4
:1015E0008A116E2201308A11BE2A3F30A6000800FF
:1015F0002508A60032303C020319302B0318302B8B
:101600008312360EF039C80037084807C900410870
:101610004902E410031DE414380EF039CA003908F9
:101620004A07CB0040084B026411031D6415E41106
:10163000E41C6419E4153A0EF039CC003B084C0761
:10164000CD003F084D026412031D6416E412E41D30
:10165000641AE416E41E712B8A112F278A15002BB9
:1016600032303C0264130319641733303C02E41334
:101670000319E4176510641FE41B651434303C0241
:10168000E5100319E5146511651CE518651535307D
:101690003C02E5110319E5156512651DE51965168E
:1016A000651E6F2B360EF039C80037084807C90091
:1016B000380EF039CA0039084A07CB003A0EF03923
:1016C000CC003B084C07CD004B088316A4008312C6
:1016D0004D088316A500831249088A11D42A3F3089
:1016E000A60008008A119E218A1188298316861671
:1016F00005108312861C7E2B63107F2B631422102F
:101700006318221422088500861E882BE310892B7B
:10171000E3142311E3182315230886008618DF013C
:101720005B08031D992BDF0A1E305F02031D992BF6
:101730000800DB0A792B8316861605108312221007
:1017400086182214220885002311861A23152308DF
:1017500086008618DF015B08031DB42BDF0A1E30EC
:101760005F02031DB42B0800DB0A9E2B83160613B1
:1017700006168312861CBE2B6310BF2B6314231323
:101780006318231723088600061EC82BE310C92BF5
:10179000E3142311E3182315230886008618DF01BC
:1017A0005B08031DD92BDF0A1E305F02031DD92BF6
:1017B0000800DB0AB92B83160613061683122313BF
:1017C00086182317230886002311061A23152308D9
:1017D00086008618DF015B08031DF42BDF0A1E302C
:1017E0005F02031DF42B0800DB0ADE2B5B100530C3
:1017F0003B0203195B1406303B02DB100319DB14B8
:101800003A1C0F2C5B18072C83160510092C831625
:10181000051483122210DB18221422088500BA1C3A
:101820001E2C5B18162C83168510182C8316851415
:101830008312A210DB18A214220885003A1D2D2C59
:101840005B18252C83160511272C8316051583128A
:101850002211DB18221522088500BA1D3C2C5B18CA
:10186000342C83168511362C831685158312A2110C
:10187000DB18A21522088500391C4B2C5B18432C61
:1018800083160512452C8316051683122212DB18C7
:10189000221622088500B91C5A2C5B18522C83167C
:1018A0008512542C831685168312A212DB18A216F9
:1018B00022088500391D692C5B18612C83160610DF
:1018C000632C8316061483122310DB1823142308B9
:1018D0008600B91D782C5B18702C83168611722C2B
:1018E000831686158312A311DB18A315230886001F
:1018F000381C872C5B187F2C83160612812C8316CC
:10190000061683122312DB18231623088600B81C40
:10191000962C5B188E2C83168612902C83168616B6
:101920008312A312DB18A31623088600381DA52CEA
:101930005B189D2C831606139F2C831606178312A3
:101940002313DB18231723088600B81DB42C5B185B
:10195000AC2C83168613AE2C831686178312A31322
:10196000DB18A31723088600BA01B901B8013A10A1
:1019700005183A14BA108518BA143A1105193A150F
:10198000BA108518BA143910051A3914B910851A05
:10199000B914391106183915B9118619B915381045
:1019A000061A3814B810861AB8143811061B3815E0
:1019B000B811861BB8150800DB01FF30DF000430CA
:1019C00092003130831692008312E301E401E601B4
:1019D0002030E7008317E801E9016D1083128C1AAB
:1019E00008008C185B178C1CF32C8C10E030DB0586
:1019F00005185B14861ADB14861B5B15061BDB15AA
:101A0000061A5B16E30A63080319DB165B085F021C
:101A10000319202D6708031D0F2DDB17EE2C203036
:101A2000660784005B088000840A63088000040A5B
:101A3000E600E703E0305B05DF00DB01E301EE2CAD
:101A40006D18362D203067020319EE2C2030640704
:101A5000840068080005EC006C086902031D322D43
:101A60006D14EE2C0230E407E70AEE2C8316981C66
:101A7000EE2C2030831267020319EE2C203064070D
:101A8000840000089900840A00089900040AE40010
:101A9000E70AEE2C8A11882083123B088A15031D61
:101AA000562D72238A1576238A15DB2D01303B02D1
:101AB000031D5F2D72238A159B238A15DB2D0230AF
:101AC0003B02031D682D72238A15B6238A15DB2D70
:101AD00003303B02031D712D72238A15DB238A1507
:101AE000DB2D04303B02031DA22D25088A11B021F5
:101AF00014308A11EE2083123A088A15031D832DB3
:101B000081308A118E2901303A02031D8A2D40301E
:101B10008A118E2902303A02031D912D20308A113C
:101B20008E2903303A02031D982D15308A118E2913
:101B300004303A02031D9F2D0A308A118E293F304E
:101B4000A600080005303B0249110319491506306B
:101B50003B02C9110319C9154912491DC919491672
:101B600007303B02C9120319C9164913491EC91A85
:101B70004917491FCF2DF62383122508A6003808E0
:101B80008A1147208312A80039088A11472083123E
:101B9000A9003A088A1147208312AA0008000A30D7
:101BA0003B02031DD82D2508A600DC248A15DB2D59
:101BB0003F30A600080083128618DF2DDB2D831628
:101BC000061740308A118E292508A600080025082E
:101BD000A6002030A8005730A9006930AA00733051
:101BE000AB007030AC003630AD003430AE00383071
:101BF000AF002030B00008002508A6000800250826
:101C0000A6002030A8003130A9002E30AA003330C1
:101C1000AB003030AC002030AD0008002708A60033
:101C200008008A11882083122508A6008A118829B5
:101C30003F30A600080007309F00A2102208850050
:101C4000A21122088500831605148510051185113F
:101C500005120614861506168616061786174030D6
:101C60008A118E218312A3132308860083168613FC
:101C70008312C201831686138A11822064308A116E
:101C80000520831686178A11882064308A11052062
:101C90008312C20A033042028A15031D3A2E8A11AA
:101CA000BF218312C5102018C5148A15C5185C2ED3
:101CB0008A11B3208A154F2E8A11CD218312C300B9
:101CC0007F304305A40024088A1123208312A50035
:101CD0002330A600463025028A150319712E0318F9
:101CE000742E2508A600E82E47302502031D7B2E02
:101CF00011268A15E82E48302502031D822EE42580
:101D00008A15E82E49302502031D8A2E8A112F27B5
:101D10008A15E82E4A302502031D912EF8228A15D5
:101D2000E82E4B302502031D982E18268A15E82E22
:101D30004C302502031D9F2EAE208A15E82E4D3013
:101D40002502031DA62EF8228A15E82E4E30250204
:101D5000031DAD2E0E268A15E82E50302502031DD8
:101D6000B42E4A258A15E82E51302502031DBB2EBC
:101D7000FC258A15E82E52302502031DC32E8A1138
:101D80005C278A15E82E53302502031DCA2E18261B
:101D90008A15E82E54302502031DD12EE7258A1519
:101DA000E82E56302502031DD82EFF258A15E82E71
:101DB00057302502031DDF2EAE208A15E82E58303D
:101DC0002502031DE72E8A116E238A15E82E182698
:101DD00001308A115020831225088A113E20831277
:0C1DE000BB0026088A11B0218A154F2E86
:02400E00423F2F
:00000001FF
